:100000000C9463030C949B030C949B030C949B0330
:100010000C949B030C949B030C949B030C949B03E8
:100020000C949B030C949B030C9423210C94F521BA
:100030000C94B11B0C949B030C949B030C949B039A
:100040000C949B030C949B030C949B030C949B03B8
:100050000C949B030C943A1C0C949B030C949B03F0
:100060000C949B030C949B030C949B030C949B0398
:100070000C949B030C949B030C949B030C949B0388
:100080000C949B030C949B030C949B030C949B0378
:100090000C949B030C949B030C949B030C949B0368
:1000A0000C949B030C949B030C949B03860686067E
:1000B000B206B20613070A080A080A0831079907A8
:1000C000AA07AA07AB151D16B3157D158115B7151F
:1000D0008415BA15C5158F1513169315C9159715DF
:1000E000CD15F7159B15D1150116A115D715E115DD
:1000F0008815BE158B15C115A615DC15ED150D1649
:100100000F167915AF152616DB17E117CF17D51780
:10011000E717ED17F317F018F3182A193D194519C9
:1001200050195319531953199B199B1958195B19D5
:1001300060196D197A197D1981198E195D22842231
:100140007C2384227C23D022F3227C234A2359233C
:100150004D004E0029003B003D003F0041004300A0
:1001600045004A004B003A003C003E00400042007F
:1001700044004C005600540035001F0021002300AD
:10018000250027002E0055002A001E002000220016
:10019000240026002D003100570060002B001A00BB
:1001A00015001C000C001300300061005F001400FB
:1001B00008001700180012002F002A0057005D00E9
:1001C000E000160009000B000E00330028005E005E
:1001D0005C00040007000A000D000F00340000005E
:1001E00058005A0052001D0006000500100037009C
:1001F000E5005B005900E1001B001900110036000A
:1002000038002152580062005100215200000000C5
:1002100000000000E700630050004F00E200000013
:100220002C000000E600E4000100010001000100D4
:1002300001000100010001000100010001000100B6
:1002400001000100010001000100010001000100A6
:100250000100010001000100010001000100010096
:100260000100010001000100010001000100010086
:1002700001000100010052002A00010001000100FC
:100280000100010001004E004E00010001000100CC
:1002900001000100010001000100510028000100DF
:1002A0000100010001000100010050004F000100A9
:1002B0000100010001000000010001000100AE008A
:1002C000AA00010001000100010001000100AC00D2
:1002D000AB00A900010001000100010001000100C4
:1002E000010001000000000000000000010001000A
:1002F00001000100010000000100000001000100F8
:1003000001000100010001000100010001000100E5
:1003100001000100010001000100010001000100D5
:1003200001000100010001000100010001000100C5
:1003300001000100010001000100010001000100B5
:1003400001000100010001000100010001000100A5
:100350000100010001000100010001000100010095
:100360000100010001000100010001000100010085
:100370000100010001000100010001000100010075
:100380000100010001000100010001000100000066
:100390000100010001000100010001000100010055
:1003A0000100010001000100010001000100010045
:1003B0000100010001000100010001000000000037
:1003C0000000000001000100010001000100000028
:1003D0000100000001000100010001000100010016
:1003E0000100010001000100010001000100010005
:1003F00001000100010001000100010001000100F5
:1004000001000100010001000100010001000100E4
:1004100001000100010001000100010001000100D4
:1004200001000100010001000100010001000100C4
:1004300001000100010001000100010001000100B4
:1004400001000100010001000100010001000100A4
:100450000100010001000100010001000100010094
:100460000100010001000000010001000100010085
:100470000100010001000100010001000100010074
:100480000100010001000100010001000100010064
:100490000100010000000000000000000100010058
:1004A0000100010001000000010000000100010046
:1004B00000000000000000002A2B280000000000BF
:1004C0000000000000000000000000290000000003
:1004D0002C1E3420212224342627252E362D373871
:1004E000271E1F202122232425263333362E37387A
:1004F0001F0405060708090A0B0C0D0E0F10111238
:10050000131415161718191A1B1C1D2F3130232D03
:10051000350405060708090A0B0C0D0E0F10111201
:10052000131415161718191A1B1C1D2F3130354CB2
:1005300000000000000000000000000000000000BB
:1005400000000000000000000000000000000000AB
:10055000000000007E0F00D4FFFFFFC700000078FE
:100560000C0341006500670069007300000012037E
:100570004100450062006F0061007200640073007A
:1005800000000403090409025B00030100A0FA094A
:1005900004000001030101000921110100012244AE
:1005A000000705810308000109040100020300009F
:1005B0000009211101000122220007058203200009
:1005C00001070503032000010904020001030000E4
:1005D00000092111010001226D000705840320009C
:1005E0000112010002000000084541070801000156
:1005F0000200010660FF0961A1010962150026FFE2
:10060000009520750881020963150026FF009520DA
:1006100075089102C005010980A101850319012A0D
:10062000B700150126B700950175108100C0050CB3
:100630000901A101850419012AA002150126A002C1
:10064000950175108100C005010906A10185060507
:100650000719E029E71500250195087501810205B4
:1006600007190029EF1500250195F0750181020594
:1006700008190129059505750191029501750391E8
:1006800001C005010906A101050719E029E71500C8
:1006900025019508750181029501750881010507FD
:1006A000190029FF150026FF009506750881000531
:1006B0000819012905150025019505750191029577
:1006C0000175039101C011241FBECFEFDAE0DEBF38
:1006D000CDBF04B603FE18C08091F2029091F302E0
:1006E000A091F402B091F5028730904BA740B04B37
:1006F00059F41092F2021092F3021092F402109246
:10070000F502E0E0F8E3099511E0A0E0B1E0E0EBEC
:10071000F8E402C005900D92AC3AB107D9F722E097
:10072000ACEAB1E001C01D92A23FB207E1F70E941E
:1007300059130C9456240C9400008430B0F46C309F
:10074000A0F4493090F49CE6899FF001112489E0DF
:10075000689FE00DF11D1124E40FF11DEE0FFF1F46
:10076000E05BFE4F85919491089581E090E00895BB
:1007700081E0089581E008950E94BA0308950E94DF
:10078000BC0308950E94BA03089508950E94C5030A
:100790000895A6E0B0E0EFECF3E00C94C6234983A3
:1007A0005A839E833091B30189819A81311115C09A
:1007B0003E81332359F0222349F00E94A009182FCB
:1007C000682F89819A810E947C0903C00E948E094A
:1007D000182F69817A81812F04C00E94A009698144
:1007E0007A810E94F9102696E3E00C94E223FC0142
:1007F000262F4081518162817381848195810E947D
:10080000C9030895CF93DF93EC0161E00E94F703E1
:10081000BE010E94BF03DF91CF910895CF93DF9374
:10082000EC0160E00E94F703BE010E94C603DF9165
:10083000CF91089591E001C0990F8A95EAF7892F29
:100840000E94C5080895CF93C82F81E00C2E01C0E7
:10085000880F0A94EAF70E944C0E8C2F0E941A040B
:10086000CF91089581E008950E9432040895CF93B6
:10087000C82F0E9477088C2F0E9434042FEF84E346
:100880009CE0215080409040E1F700C00000CF91F3
:10089000089581E00E9437040E94601C089580E062
:1008A0000E9437040E94841C08950F931F93CF93D6
:1008B000DF938C0161E00E94F703EC01B8010E9414
:1008C000BD18882309F457C0B801CE010E94C203A5
:1008D000882309F450C0B801CE010E94C3178823B1
:1008E00009F449C0B801CE010E945515882309F4C6
:1008F00042C0B801CE010E942B158823E1F1B80156
:10090000CE010E9406188823B1F1B801CE010E94E1
:10091000F711882381F1F8018581882341F1C330E3
:100920008CE7D807D1F040F4C115FCE7DF0791F060
:10093000C130DC47A1F01BC0CB35ECE7DE07A9F0E6
:10094000CC35FCE7DF0771F0CA35DC4781F40E9443
:10095000270E0DC00E9449040EC00E942F0E0E9457
:100960004F0409C00E941D0E02C00E942B0EC80138
:100970000E94B80301C080E0DF91CF911F910F91D9
:1009800008950E94891B0E94E10408950E94E504D5
:100990000E94921B089581E008950895CF93DF93FC
:1009A000D82F0E94CB04C82F882319F08D2F0E94C6
:1009B000CD048C2FDF91CF91089508950E94CE042D
:1009C000089580E00E94DE0408950E94AB190E9401
:1009D000DE040895CF930E94AB19C82F8091AE0119
:1009E000C81779F0C093AE010E941F1C6093AF013D
:1009F0007093B0018093B1019093B2018C2F0E944B
:100A0000DE04CF910895ADE0B0E0E9E0F5E00C94AC
:100A1000C723488759876A877B878C879D87911171
:100A20000E94290DCE01019627E0FC0111922A9522
:100A3000E9F726E0FE013896DC0101900D922A9537
:100A4000E1F72D8121110AC029813A814B815C8116
:100A50006D817E818F810E94730C04C00E9402040C
:100A60008111F2CF2D96E2E00C94E323FC01248166
:100A7000213021F4808191810E94CD090895CF9386
:100A8000882309F47FC0C82F8238A1F40E94B819C6
:100A900081FD78C089E30E94CB1A0E94B00D2FEF30
:100AA00087EE93E0215080409040E1F700C00000C5
:100AB00089E315C08338C1F40E94B81980FD62C073
:100AC00083E50E94CB1A0E94B00D2FEF81EE94E0D7
:100AD000215080409040E1F700C0000083E50E9473
:100AE000E51A0E94B00D4EC08438A1F40E94B819D6
:100AF00082FD48C087E40E94CB1A0E94B00D2FEF00
:100B000081EE94E0215080409040E1F700C0000069
:100B100087E4E5CF8CEF8C0F813A70F48C2F0E9424
:100B2000401A882329F08C2F0E94E51A0E94B00DEC
:100B30008C2F0E94CB1AD5CF80E28C0F883048F4DE
:100B4000C77081E001C0880FCA95EAF70E940C0DBA
:100B5000C8CFEBE5EC0FE33040F4F0E0E55BFE4F8F
:100B6000808190E00E94D4190DC0C85ACB3150F456
:100B7000EC2FF0E0EE0FFF1FEB5EFE4F80819181C6
:100B80000E94F919CF910895882309F44DC0823845
:100B900059F40E94B81981FF47C089E30E94CB1A1B
:100BA0000E94B00D89E30CC0833879F40E94B81913
:100BB00080FF3AC083E50E94CB1A0E94B00D83E506
:100BC0000E94E51A0E94B00D0895843859F40E94DD
:100BD000B81982FF29C087E40E94CB1A0E94B00D89
:100BE00087E4EECF9CEF980F913A50F390E2980F84
:100BF000983050F4877091E001C0990F8A95EAF718
:100C0000892F0E94120DDECF9BE5980F933028F4B8
:100C100080E090E00E94D4190895885A8B3120F426
:100C200080E090E00E94F91908951F93CF93DF931D
:100C3000182FEB010E943F05209741F08FE99FE0BC
:100C40000197F1F700C000002197F6CF812F0E9495
:100C5000C405DF91CF911F910895893319F060E0A9
:100C600070E002C060E570E00E94150608958823D8
:100C700021F00E940C0D0E94B00D0895882321F0F0
:100C80000E94120D0E94B00D0895A0E0B0E0EBE4C8
:100C9000F6E00C94C1237C01162FC72FFC01D581EF
:100CA000068102950F700E94020D8823F9F0DD2362
:100CB000E9F08C2F807F803461F080E2810F8830F2
:100CC000A8F08C2F807E803221F4123078F000233F
:100CD00069F08091B00282FF09C082E00E94F10DAC
:100CE0000E94020D91E0D82ED92601C0D12CCC2E25
:100CF000C2948FE0C8228C2D90E08C30910508F0D2
:100D000089C1FC01EA5AFF4F0C94AA238C2F807FE3
:100D1000CF70882311F0C295C07FDD2399F0CC23DA
:100D200009F464C180E2810F883010F0111104C011
:100D30008C2F0E940C0D03C08C2F0E941C0D0E9452
:100D4000B00D54C1812F0E94C405CC2309F462C1A7
:100D500080E2810F883038F1112329F18C2F0E9415
:100D6000220D24C08C2F807FCF70803211F0C2956D
:100D7000C07F112319F0113099F13CC08091B0026D
:100D800082FD17C0DD2349F0CC2329F08C2F0E946F
:100D90000C0D0E94B00D80E02AC180E00E94C405C5
:100DA000CC2309F437C18C2F0E94120D0E94B00D84
:100DB00031C1DD2349F0002309F1013009F02AC1D6
:100DC0008C2F0E94330D26C1011124C18C2F0E944B
:100DD0003E068C2F0E943F0D8C2F0E94C40D1AC11D
:100DE000DD2321F0063008F015C108C0053008F0F9
:100DF00011C115C0DD2331F00111F8C08C2F0E9404
:100E0000370608C1002359F0193309F000C1FFEF7C
:100E100027EE83E0F15020408040E1F7F6C08C2FB0
:100E20000E943E06F7C08C2F86958695837019F038
:100E3000813061F0EFC0DD2321F0812F9C2F937072
:100E400002C080E090E00E94D419ECC0DD2321F0C4
:100E5000812F9C2F937002C080E090E00E94F919CE
:100E6000E1C08C2F837079F5D111D8C0412F429504
:100E700046954770440F440F212F2F70042E01C058
:100E8000220F0A94EAF714FF08C08FE090E001C037
:100E9000880F4A95EAF7809501C080E0C695C6950F
:100EA000C370822BC23049F058F4C13019F00E944F
:100EB000CE08B4C00E94C808B1C00E94D408AEC019
:100EC0000E94C508ABC0DD2319F08C2F817001C0D2
:100ED0008695882309F4A2C0412F42954695477014
:100EE000440F440F212F2F70042E01C0220F0A94AB
:100EF000EAF714FF08C08FE090E001C0880F4A9520
:100F0000EAF7809501C080E0C695C695C370822B34
:100F1000C23049F058F4C13019F00E941A097EC05D
:100F20000E9414097BC00E94200978C00E94DD083D
:100F300075C0CF70DD2339F08C2F0E94EF08812F10
:100F40000E9437066BC0812F0E943E068C2F0E94A4
:100F5000FB0864C0123F21F128F4103F41F0113F1B
:100F6000C1F040C0133F19F1143F79F03BC0DD23BD
:100F700041F0053008F04EC08C2F8F710E94080997
:100F800049C0063008F046C0F7CF8091B00282FD1C
:100F900018C0DD2339F08C2F8F710E94EF083AC002
:100FA000DD23C9F38C2F8F710E94FB0833C0DD2332
:100FB00029F08C2F8F710E94E6082CC00E94E20855
:100FC00029C0DD2331F063E08C2F8F710E94D30D97
:100FD00021C081E00E94F10D0230E0F082E00E9429
:100FE000F10D18C0DD2331F00023A9F2812F0E94FA
:100FF0003F0510C00023B1F2193349F49FEFE7EE2B
:10100000F3E09150E040F040E1F700C00000812F94
:101010000E94C40588EF8C0D843020F40E94AB1927
:101020000E94DE04DD2089F00E94FE0C80FD0DC0D0
:10103000F70115820E94F80C0E94EF08C7010E9478
:1010400042080E94F80C0E94FB08CDB7DEB7E8E02A
:101050000C94DD230F931F93CF93DF93EC016881F2
:1010600079818D810E94D8098C010E9426090E94F5
:10107000B808B801CE010E944506DF91CF911F91BB
:101080000F910895CF93DF93FC0124812223D1F0A7
:10109000EC010E94550481110FC00E94020D8823AB
:1010A00089F08D81882371F08091B00282FF0AC09F
:1010B00082E00E94F10D06C0CE010E942A08CE01F6
:1010C0000E940E04DF91CF91089580E090E00E948D
:1010D000D41980E090E00E94F9190E94290D0E9425
:1010E000B00D08950E94FF1A0E94650808950E949D
:1010F000190D0E947208089592959F70963079F0AC
:1011000010F4925001C09A50923068F4803F69F018
:1011100018F4883E40F409C0843F29F406C0883E94
:1011200020F0813F11F080E0089581E00895FC01F6
:101130002481222339F0808191810E94CD090E946F
:101140007C08089580E00895A6E0B0E0EAEAF8E0BF
:101150000C94C7232696E2E00C94E323A7E0B0E0CA
:10116000E4EBF8E00C94C7232796E2E00C94E32329
:10117000089508950E94B90808950E94BA08089534
:101180000E94BD088093DF0108950E94C008089561
:101190009091DF01892B0E94C00808959091DF0192
:1011A00089230E94C00808959091DF0189270E9439
:1011B000C00808950E94B90808950E94DA08809333
:1011C000DE01089580E00E94DD08089591E001C0ED
:1011D000990F8A95EAF7892F0E94DD08089521E08A
:1011E00030E001C0220F8A95EAF78091DE01822B60
:1011F0000E94DD08089521E030E001C0220F8A95A9
:10120000EAF720958091DE0182230E94DD0808958F
:1012100021E030E001C0220F8A95EAF78091DE01DB
:1012200082270E94DD0808959091DE01892B0E949B
:10123000DD0808959091DE0189230E94DD0808955C
:101240009091DE0189270E94DD0808950895962F68
:101250009770A1E001C0AA0F9A95EAF793E07695FE
:1012600067959A95E1F7FB01EE0FFF1F6E0F7F1F49
:10127000FA01E60FF71F40E050E0682F70E0908120
:101280009B01042E02C0369527950A94E2F721703F
:10129000219529272A23292721934F5F5F4F433028
:1012A000510569F708959B01782F777043E0969573
:1012B00087954A95E1F7FC01EE0FFF1F8E0F9F1FE8
:1012C000F901E80FF91F40E050E080E0219130E0A3
:1012D000072E02C0369527950A94E2F7217033272E
:1012E000042E01C0220F0A94EAF7822B4F5F5F4F52
:1012F0004330510559F70895282F9C3070F48930F8
:1013000060F4862F622F70E029E0929F600D711DBE
:10131000112444EB51E00E94270908959C3070F499
:10132000893060F4292F90E064EB71E039E0239F6D
:10133000800D911D11240E945309089580E00895A5
:10134000CF92DF92FF920F931F93CF93DF936C01A5
:101350000091DE018091DF01082BC3E0D0E010E0B6
:10136000C8010C2E02C0959587950A94E2F780FD7E
:1013700004C02197A8F7F12C07C0FC2EB6018C2FD2
:101380000E9405110197A9F38F2DDF91CF911F9135
:101390000F91FF90DF90CF900895CF93DF93EC01F2
:1013A0000E94A009BE010E940511DF91CF9108950E
:1013B0001F93CF93DF93EB019091B301992321F019
:1013C000CB010E94CD0913C0882349F0CB010E94B4
:1013D000A009182F682FCE010E947C0904C0CB0100
:1013E0000E948E09182FBE01812F0E940511DF91E6
:1013F000CF911F910895E1E0F0E0DF0102C0AA0F54
:10140000BB1F6A95E2F7BD01DF0102C0AA0FBB1F37
:101410004A95E2F7AD01462B01C0EE0F2A95EAF797
:10142000942F9823491302C08E2B0895E0958E23A4
:101430000895242F462F682F8091DE010E94FB091A
:101440000E94DD0808951F93CF93DF93C091E001C0
:1014500017E08091E101C817A1F0D0E01C9FF001D6
:101460001D9FF00D1124EE51FE4F208131814281EC
:1014700053816481758186810E94AE082196C77070
:10148000E8CFDF91CF911F91089520911A023091FA
:101490001B0240911C0250911D0260911E0270912E
:1014A0001F02809120020E94AE080895CF93DF931F
:1014B0008091200282958F7009F04EC080911F02AA
:1014C000882309F449C08091E0014091E1015091E5
:1014D0001B0260911A02C0911C02D0911D0277E09C
:1014E0008417D1F190E0789FF001799FF00D1124DD
:1014F000DF01AE51BE4F14962C911497222349F16F
:1015000011962C911197251324C02C91261321C0DC
:1015100015962C91159721111CC012962D913C9176
:1015200013972C1B3D0B283C310598F48091200229
:101530008F70806180932002E851FE4F80818F7010
:10154000806180838AE192E00E9442080E94230A1F
:1015500003C001968770C4CFDF91CF910895209189
:10156000E0019091E10157E02917A9F030E0529F86
:10157000F001539FF00D1124EE51FE4F718176134F
:1015800006C07081781303C07581741306C02F5F85
:101590003F4F2770E9CF80E0089581E00895A4E1EE
:1015A000B0E0E5EDFAE00C94BD238C0186E0F80193
:1015B000DE011F9601900D928A95E1F7F801848172
:1015C000E5809AE1A92E92E0B92E90911E02911128
:1015D00018C0882309F480C1EE20D9F1C8010E9407
:1015E0009708F82E8823A9F187E0F801D50101902A
:1015F0000D928A95E1F7C5010E9436050E94560AB0
:1016000098C0F801C080D18082809380F0901F0242
:1016100020911C0230911D02A401421B530BFF209C
:1016200009F406C1483C510508F0AFC0882309F40D
:1016300055C180912002282F207F90911B022223E8
:1016400061F09D1509F462C0C8010E9497088111DC
:1016500073C0C8010E9442083FC19D1115C09091FE
:101660001A029C1111C0E1100FC08F70806180932D
:1016700020020E94450A8AE192E00E94420880917D
:101680002002F801868326C1E1103AC040E06D2DAA
:101690008C2D0E94AF0A40E06D2D8C2D0E94AF0A68
:1016A000E82E811117C1CF86D88A8F8598890E942C
:1016B000CD09292F22952F70243020F49F702230DD
:1016C00028F009C02A50223080F014C0992349F034
:1016D000811107C013C0992321F0F8019681907FF2
:1016E00069F0805E883030F409C0803F38F0815F57
:1016F000833020F0C8010E944208EF2CFE2CEEC07F
:1017000080912002816080932002E4C090911A02AF
:101710009C119ACFE11098CFF8018683C8010E94EE
:10172000420887E0F801AAE1B2E001900D928A95A3
:10173000E1F70E94450AD2C0EE2009F48ACF209139
:101740002002822F82958F7090E002978CF080911A
:101750001A0290911B02998788879B868A868091BE
:101760001E028C871D862E87CE0108960E94420895
:1017700087E0F801AAE1B2E001900D928A95E1F7C5
:101780000E94560A0E94450AA7C090912002292F64
:10179000207FA1F4682D9A8A898AA6017A899E2DD4
:1017A0000E94A4088AE192E00E94420887E0F501C5
:1017B00011928A95E9F70E94450A8CC0882309F4A2
:1017C0008DC080911B028D1111C080911A028C1165
:1017D0000DC0E1100BC0F8019683C8010E944208B9
:1017E00087E0F50111928A95E9F778C0C8010E9457
:1017F0009708882309F42DCFEE2009F42ACF2091F1
:101800002002822F82958F7090E002970CF4B0CF67
:1018100080911A0290911B029A8389839C828B8209
:1018200080911E028D831E822F83CE0101969ECF52
:10183000483C510508F040C0882309F44DC0FE2CF7
:10184000EE2009F406CF80911B028D1127C08091F4
:101850001A028C1123C09091200290FD16C0892F8E
:1018600082958F70282F30E02115310571F0F80135
:1018700096832F30310509F451CF8F5F982F9295C1
:10188000907F86818F70892B48CF87E0F801AAE18D
:10189000B2E001900D928A95E1F720C0C8010E9444
:1018A0009708811165CF809120028160809320028A
:1018B000C8010E94420812C0682D9A8A898AA6012E
:1018C0007A899E2D0E94A40887E0F50111928A95DD
:1018D000E9F72FCFF12C02C0FF24F3948F2D6496EB
:1018E000ECE00C94D923AEE0B0E0E9E7FCE00C9426
:1018F000C623288739874A875B876C877D878E87D1
:10190000CE0108960E94CF0A882361F06C85662379
:10191000A9F1288539854A855B857D858E850E945C
:10192000AE082CC087E0FE013896DE0111960190CA
:101930000D928A95E1F76C85662301F12091E10112
:1019400030E0C9010196877099274091E00150E08D
:1019500084179507E1F16D8397E0929FD001939FE3
:10196000B00D1124AE51BE4FFE01319601900D9283
:101970009A95E1F78093E1010E94230A17E0809194
:10198000E0019091E101891779F1189FC0011124BC
:101990008E519E4F0E94CF0A882331F1E091E001E1
:1019A0001E9FF0011124EE51FE4F208131814281B2
:1019B00053816481758186810E94AE088091E00127
:1019C00090E00196877099278093E001D8CF0E941C
:1019D00077081092E1011092E001EAE1F2E087E07D
:1019E000DF011D928A95E9F72E96E3E00C94E2233D
:1019F0008091490286958695869508958091490241
:101A00008770089590914902977081E009F480E011
:101A1000089580917502089590917502892B8093A5
:101A200075020895809590917502892380937502BF
:101A3000089510927502089590917402892B8093F5
:101A400074020895809590917402892380937402A2
:101A5000089510927402089508950E942C0D08951F
:101A60000E942D0D089590914B02292F2823821753
:101A700029F0982B90934B020E94300D089590917D
:101A80004B02292F282331F08095892380934B0224
:101A90000E94300D089580914B02882329F0109206
:101AA0004B0280E00E94300D0895CF93C0917502E3
:101AB00080917402C82B80914B02882331F0C82B8F
:101AC0000E941E1A81110E944B0D8C2FCF910895F8
:101AD000CF93DF93C0910201D09103010E94550D75
:101AE0008883C0910201D091030148E050E061E495
:101AF00072E0CE010E94EE23892B59F088E0FE01AE
:101B0000A1E4B2E001900D928A95E1F7CE010E9426
:101B1000BB19DF91CF910895CF93DF93C09100015E
:101B2000D09101010E94550D8983C0910001D0918F
:101B3000010140E250E061E272E0CE010E94EE233A
:101B4000892B59F080E2FE01A1E2B2E001900D92F2
:101B50008A95E1F7CE010E94C619DF91CF910895D1
:101B60000E94621B813039F48091AF0287FF03C06D
:101B70000E948C0D08950E94680D08950E942C0DFE
:101B800008950E94BE0D089590914A02292F28239E
:101B900031F08095892380934A020E94C10D0895F7
:101BA0000E942C0D08959091B00292FF11C098E010
:101BB000899F90011124262B209349020E94EF084F
:101BC000809149028695869586950E94D00D08954C
:101BD0000E94EF0808951092490280E00E94D00D03
:101BE0000895909149028095892380934902282F76
:101BF000277069F4981759F09091B00292FF07C0CE
:101C00008695869586950E94FB080E94EB0D0895A7
:101C10009091B00292FB222720F9281769F080FBEF
:101C200092F99093B0028091AF029091B0020E941D
:101C3000570E82E00E94F10D08958091B00282FB60
:101C4000882780F991E089270E94080E089581E095
:101C50000E94080E089580E00E94080E08956FEF1C
:101C60007FEF80E090E00E944024089580E090E0C3
:101C70000E940C24853E9E4F19F40E94511808952D
:101C800080E0089582E090E00E940424089583E0BB
:101C900090E00E9404240895682F83E090E00E9461
:101CA0002224089584E090E00E940C240895BC0151
:101CB00084E090E00E9440240895AB01BC018FE0D5
:101CC00090E00E9434240895AB01BC0183E190E0D0
:101CD0000E943424089560E070E0CB010E94640EFD
:101CE000089560E070E0CB010E945D0E0E946B0ED3
:101CF0000895A8E0B0E0EFE7FEE00C94C72365EE9E
:101D00007EEF80E090E00E94402460E082E090E07E
:101D10000E94222481E08093DF010E944C0E60E04B
:101D200074E184E090E00E94402460E086E090E06E
:101D30000E94222460E087E090E00E94222440E09C
:101D400050E0BA0188E090E00E94342460E083E231
:101D500090E00E94222460E08CE090E00E94222427
:101D600060E08DE090E00E94222419821A821B829A
:101D70001C821D821E821F82188648E050E067E1A7
:101D800070E0CE0101960E94122440E050E0BA01BA
:101D90008FE190E00E94342480E00E946A180E9443
:101DA0009F180E94710E2896E2E00C94E3230E9493
:101DB000790E0895682F8EE090E00E942224089505
:101DC000A6E0B0E0E6EEFEE00C94C5230E94131CF2
:101DD0008C0180917602909177020817190781F0A3
:101DE00019821A820E94131C682F49815A81792F07
:101DF00080E090E00E940305109377020093760242
:101E00002696E4E00C94E1230E941F1C6093940248
:101E1000709395028093960290939702609390023C
:101E2000709391028093920290939302089581E0BF
:101E3000089581E008950E94190F089508950E9461
:101E40001E0F08950E941E0F08950E94220F0895EC
:101E50000E941E0F08950E94280F08950E941E0FD1
:101E6000089585EF91E10E9470130E942E0F0E9449
:101E70002B0F08950E941F0F0E941E0F08950E94AD
:101E8000360E811102C00E94D70E0E94420E80932E
:101E900098020E94520E9093B0028093AF020E946B
:101EA00093130E94470E0E94C5088091DE010E9494
:101EB000DA0808950E940A1C0E94AF180E94C812F6
:101EC0000E943F0F0E94DD040E94250F0895A6E0A6
:101ED000B0E0EDE6FFE00C94BB230E94170F8111E8
:101EE00003C00E94E00E62C00E94DE1228E7E22ECC
:101EF00022E0F22E5701D12CF501019111915F01E1
:101F00008D2D0E940A1280279127D394FCE0DF16C2
:101F100019F0892B89F302C0892B19F3809198025B
:101F200081FD0E9413120E941B0F782E10E0662480
:101F30006394812F0E940A124C01F701A080B180A6
:101F4000A826B926A114B10449F100E0CC24C39419
:101F5000D12CC5018C219D21892BC1F07720B1F0B6
:101F600009831A830E94131C9C838B836D8221E05A
:101F7000C4018C219D21892B09F420E049815A81DB
:101F80006B817C818D81922F0E9403050F5FCC0CA9
:101F9000DD1C0930F1F6F701918280821F5FF2E0CB
:101FA000EF0EF11C1C3029F60E94040F0E94EA0477
:101FB0002696EEE00C94D7231F93CF93DF930E94D5
:101FC0000A11EC01C11580E5D807E8F5C11590E4C8
:101FD000D90708F0A8C0C03ED10530F5CD3CD105E9
:101FE00008F094C0C83AD10578F4C53AD10508F094
:101FF00083C0C130D10509F47CC008F4F2C0C430FC
:10200000D10508F0F1C0EDC0C33CD10508F0E9C02E
:10201000C85AD0E0CC0FDD1FC25BDE4F0990D881DB
:10202000C02DCE019464E1C0C11580E2D80708F04C
:10203000CBC0C11591E0D90708F06BC0C83ED105EF
:1020400008F4D2C0CEC0C03682E5D80728F5C03427
:1020500092E5D90708F079C0C03282E5D80708F0C8
:102060006CC0C11592E5D90708F481C04C2F469584
:10207000469580E2489FA0011124C37021E030E022
:10208000C90102C0880F991FCA95E2F7EA01C82B5F
:10209000D92BCE019D68A9C0C03A82E5D807B8F413
:1020A0008C2F8F71C03892E5D90708F07BC08695D8
:1020B000869590E2899F90011124C37081E090E0A1
:1020C00002C0880F991FCA95E2F79A6868C0C03CA1
:1020D00082E5D80708F46DC0C03E92E5D90708F044
:1020E00080C0CF71DD27DC2FCC27CE01806F906AB6
:1020F0007CC081E090E079C0C55AD0E0CC57DE4F7B
:102100008881C82FD0E0CE0190646FC0CE01906569
:102110006CC08D2F0E94A611182FCE0199270E9406
:102120000A111F715CC0CE0199270E940A11CC27A9
:10213000DF70D06A8C2B9D2B58C0CF71D0E0DC2F84
:10214000CC27CE01816F906A50C08C2F8F718695FD
:10215000869590E2899F90011124C37081E090E000
:1021600002C0880F991FCA95E2F79C6818C08C2F8F
:102170008F710E94A61195E0D695C7959A95E1F7C3
:10218000CF70D0E0DC2FCC27282F30E084FF05C0B3
:1021900084E0220F331F8A95E1F7D069CE01822BAC
:1021A000932B23C090E0D82FCC27CE01846F906A68
:1021B0001CC08C2F8F710E94A6118F7190E0D82FB8
:1021C000CC27CE01906211C08D2F8F710E94A61175
:1021D000182FCE0199270E940A111F719062912B2E
:1021E00004C080E090E001C0CE01DF91CF911F914B
:1021F00008957C3038F4693028F4462F672F0E9408
:102200004514089580E090E008950E94F9100E941E
:10221000DC0F08958238910569F1B0F4813391059E
:1022200009F475C048F48932910509F467C08A320F
:10223000910509F471C008958533910509F459C0D9
:1022400089339105B9F00895833E910589F138F4F9
:10225000803E9105D1F0823E910529F10895863E98
:102260009105C9F1873E9105D9F1843E910509F0A8
:102270006CC027C02091AF0220FD57C021FD55C082
:102280002091B00223FD5BC008958091AF0280FDD4
:1022900048C08091B00280FF48C08091AF0284FDA9
:1022A00046C083EE51C08091AF0282FF3CC0F5CFA3
:1022B0008091AF0282FD37C08091B00280FD35C0B1
:1022C000ECCF8091B00281FF36C08091AF0284FDD7
:1022D0002EC087EE39C08091AF0283FF2AC0F5CFB0
:1022E0008091AF0283FD25C08091B00281FD23C0A3
:1022F000ECCF8091AF0285FD22C01FC08091AF025C
:1023000085FD1BC08091B00283FF19C00AC0809177
:10231000AF0286FD16C017C08091AF0286FD13C0C4
:1023200010C089E311C082EE0FC080EE0DC080E0C6
:102330000BC086EE09C084EE07C085E305C089E2C4
:1023400003C08AE201C081E390E008959091AF025A
:1023500092FF10C041E0282F2471243009F040E0A2
:1023600031E0282F2871283009F030E0431711F0B0
:102370002CE0822793FF10C041E0282F24712431E4
:1023800009F040E031E0282F2871283109F030E0D1
:10239000431711F02CE082273091B00230FF10C0BB
:1023A00051E0282F2171213009F050E041E0282F21
:1023B0002871283009F040E0541711F029E08227F5
:1023C00031FF10C041E0282F2171213109F040E098
:1023D00031E0282F2871283109F030E0431711F03F
:1023E00029E0822794FD877E089580E00895CF93A9
:1023F0009C01205E32452032310540F4FB01C5814D
:10240000C11105C08F710E94230401C0C1E08C2F4F
:10241000CF910895E82FF0E0EE0FFF1FE753FD4F37
:10242000808191810895089580EA8A95F1F7089551
:1024300000C008950E941412089508950E941D126C
:1024400008950E941E1208950E941D1208950E9470
:1024500024120895F894E82FE295EF70F0E031A18E
:10246000282F2F7081E090E001C0880F2A95EAF7AD
:10247000982F9095932391A392A1892B82A378946E
:1024800008950F931F93CF93DF93C0E9D1E0899113
:102490008F3F11F00E942A1281E0CC39D807B9F79A
:1024A000C7E8D1E000E911E089918F3F11F00E9467
:1024B0002A120C171D07C1F7DF91CF911F910F91C1
:1024C0000895A0E0B0E0E7E6F2E10C94C0238C01AF
:1024D000C62FD0E0CE0180579E4F6C01FC01908149
:1024E0009F3F09F450C0B62EF894E92FE295EF70A3
:1024F000F0E081A19F7021E030E001C0220F9A95A9
:10250000EAF7822B81A382A12095282322A3789425
:102510000E941812E7E8F1E040E951E021E030E0E4
:10252000E12CF12C61916F3F89F0A62FA295AF703D
:10253000B0E090968C9190E06F7002C09595879571
:102540006A95E2F780FD02C0C90102C080E090E018
:10255000E82AF92A220F331F4E175F0719F7F601F1
:1025600080818F3F11F00E942A1261E0E114F10492
:1025700009F460E08B2D0E941A12CC0FDD1FC00FF2
:10258000D11FF982E882CDB7DEB7E9E00C94DC23F5
:102590000E94411288E1E9ECF2E0DF01982F1D92E0
:1025A0009A95E9F7E1EBF2E0DF011D928A95E9F7F0
:1025B0008CE00E9419130E9427120895A8E1B0E050
:1025C000E4EEF2E10C94C4238E010F5F1F4F88E10B
:1025D000F80111928A95E9F7F12C6F2DC8010E943C
:1025E0006112F394FCE0FF12F8CF48E150E0B8012B
:1025F00081EB92E00E94EE2321E0009709F420E0B5
:10260000892B41F088E1F801A1EBB2E001900D9235
:102610008A95E1F74CE069EC72E081EB92E00E9470
:102620001A13182F0E942112812F6896E5E00C944E
:10263000E0230895EF92FF920F931F93CF93DF93C0
:102640007C018B01C42F222351F081E080939B02F7
:102650000E94131C90939A028093990204C0809167
:102660009B02811102C080E01CC080919902909170
:102670009A020E942B1C0597B0F3D0E0CC0FDD1F0F
:10268000AE01B701C8010E94EE23892B39F0AE01DB
:10269000B701C8010E94FB2381E001C080E01092D5
:1026A0009B02CDB7DEB7E6E00C94DF230E94670FF4
:1026B00008950E94AA1B0E941C1E0E94310F0E94B6
:1026C000361E0E945A0F0E94431E0E94481E0E94FE
:1026D00056130E94621E0E94E11C0E943A0FF5CF21
:1026E0009093AD018093AC0108950E942F0E089540
:1026F00080E00E940A12817008950E94DE122FEF7E
:1027000086E791E0215080409040E1F700C0000052
:102710000E94DE120E947813882321F00E94751314
:102720000E94601C08950E947D13089584E008951E
:1027300050E0440F551F22E1629F400D511D1124AE
:102740009A0168ED869F200D311D1124C9018896DC
:1027500008950F931F93CF93DF938430A0F46C30D0
:1027600090F4493080F40E9498138C010E94042454
:1027700090E0D82FCC27C80101960E9404249E0126
:10278000282BC90102C080E090E0DF91CF911F911A
:102790000F9108950F931F93CF93DF93843080F4AC
:1027A0006C3070F4493060F4E9010E9498138C0198
:1027B0006D2F0E9422246C2FC80101960E942224B2
:1027C000DF91CF911F910F9108951F93CF93DF93C6
:1027D000D0E0C0E010E0412F6C2F8D2F0E949D03B0
:1027E0009C01412F6C2F8D2F0E94CA131F5F19303F
:1027F00091F7CF5FCC3071F7DF5FD43051F7DF91C5
:10280000CF911F910895EF92FF920F931F93CF9353
:10281000DF93EA017A01E60EF71E8C01C801889663
:10282000CE15DF0569F0003623E0120720F40E9480
:102830000424888301C0188221960F5F1F4FEECFBA
:10284000CDB7DEB7E6E00C94DF23EF92FF920F9353
:102850001F93CF93DF93EA017A01E60EF71E8C01F6
:10286000C8018896CE15DF0559F0003623E012071F
:1028700018F468810E94222421960F5F1F4FF0CF29
:10288000CDB7DEB7E6E00C94DF23843038F46C304B
:1028900028F4493018F40E94A913089580E090E0CC
:1028A000089580E1089588E790E00895EF92FF92FF
:1028B0000F931F93CF93DF93EA017A01E60EF71E81
:1028C0008C01C80188579C4FCE15DF0561F0083791
:1028D000110520F40E940424888301C018822196E7
:1028E0000F5F1F4FEECFCDB7DEB7E6E00C94DF23CE
:1028F000EF92FF920F931F93CF93DF93EA017A0138
:10290000E60EF71E8C01C80188579C4FCE15DF05D7
:1029100051F00837110518F468810E94222421968D
:102920000F5F1F4FF0CFCDB7DEB7E6E00C94DF238B
:10293000CF93DF93C8E8D3E060E0CE010E94222469
:102940002196C11584E0D807B9F7DF91CF9108959A
:10295000A8E0B0E0EEEAF4E10C94BD23F82E8FE09D
:102960008F1508F474C08FEF93E00E940424811146
:102970006EC008E813E0FF2071F0011594E019071C
:1029800009F465C0C8010E940424811101C0FA94B1
:102990000F5F1F4FF0CFFE0131966F0188E011925B
:1029A0008A95E9F77801FFEFEF1AFF0AC8010E9444
:1029B000042489831A82882309F449C0813009F0EC
:1029C00040C0580182E0A80EB11CC7010E94042437
:1029D0008A838823E1F19FEF980F933060F47801A8
:1029E00093E0E90EF11CC5010E9404248B83882327
:1029F00071F11C8226C0843019F54E01E3E08E0E81
:102A0000911C02E010E07501FFEFEF1AFF0AC5010B
:102A10000E940424F40181934F018823C1F08C3774
:102A200041F4E2E0F0E0EC0FFD1FE00FF11F108237
:102A300008C00F5F1F4F57010730110521F707C06E
:102A4000750160E0C6010E94F1168701ABCF2896A0
:102A5000ECE00C94D923CF93DF9386319C4709F5A2
:102A6000EB010E94090D9D81992371F08A7A91E012
:102A700009F490E090939C02811102C089E201C0A8
:102A800085E30E94CB1A09C080919C02811102C08B
:102A900089E201C085E30E94E51A0E94B00D80E042
:102AA00001C081E0DF91CF910895CF93DF93FC01C6
:102AB000DB0115968C91882309F4DDC09F01305706
:102AC0002332310508F0D8C0EF010E94520E9093D6
:102AD000B0028093AF02FE01E150F047E232F1050F
:102AE00020F4EE59FF4F0C94AA238091AF0281602D
:102AF000AAC08091B0028860B2C08091AF028260AB
:102B0000A2C08091AF0220C08091AF0288609BC0BC
:102B10008091B0021EC08091B0028260A0C08091FE
:102B2000AF02806190C08091AF0280628CC08091C2
:102B3000AF02806488C00E9477088091AF028068ED
:102B400082C08091AF02886084607DC08091B002B5
:102B50008260816084C08091AF028E7F74C080915A
:102B6000B002877F7CC08091AF028D7F6CC0809166
:102B7000AF0220C08091AF02877F65C08091B00214
:102B80001EC08091B0028D7F6AC08091AF028F7E9F
:102B90005AC08091AF028F7D56C08091AF028F7B6B
:102BA00052C00E9477088091AF028F774CC080910D
:102BB000AF02877F8B7F47C08091B0028D7F8E7F71
:102BC0004EC08091AF0282FB222720F991E092272C
:102BD00090FB82F990FB83F936C08091B002982F68
:102BE000909591708E7F892B90FB81F938C08091F0
:102BF000AF0286FB222720F991E0922790FB86F90D
:102C000022C00E9477088091AF0287FB222720F91B
:102C100091E0922790FB87F916C081E001C080E027
:102C20000E94DA0E1EC08091AF0284FB222720F999
:102C300091E0922790FB84F906C08091AF02982F13
:102C4000909590FB80F98093AF020BC08091B00209
:102C500083FB222720F991E0922790FB83F9809350
:102C6000B0028091AF029091B0020E94570E0E9474
:102C7000770880E001C081E0DF91CF9108958F92C5
:102C80009F92BF92CF92DF92EF92FF920F931F938A
:102C9000CF93DF93E82FF0E0E055FB4FB490282F5F
:102CA00026952695269530E0F901E05BFA4FE490F1
:102CB0008770F12C082E02C0F594E7940A94E2F78D
:102CC00091E0E922FF24F901E05CFA4FC490D12C95
:102CD000082E02C0D594C7940A94E2F7E1E0CE2210
:102CE000DD24F901E05DFA4FC491D0E002C0D59532
:102CF000C7958A95E2F7C170DD27062F10E0E11431
:102D0000F10471F081EE0E943F05C801009741F087
:102D1000EFE9FFE03197F1F700C000000197F6CF2F
:102D2000C114D10439F44801B8018B2D0E94150655
:102D3000C8010EC086EE0E943F05C801009799F3B6
:102D4000EFE9FFE03197F1F700C000000197F6CFFF
:102D5000009741F0EFE9FFE03197F1F700C0000084
:102D60000197F6CFCD2819F5EF2879F081EE0E9472
:102D7000C4050115110549F08FE99FE00197F1F7AE
:102D800000C0000001501109F4CFCD2BF1F08CE20E
:102D90000E942D0681149104C1F0EFE9FFE0319704
:102DA000F1F700C00000F1E08F1A9108F3CF86EE32
:102DB0000E94C405C8010097B9F2EFE9FFE031971E
:102DC000F1F700C000000197F6CFDF91CF911F917E
:102DD0000F91FF90EF90DF90CF90BF909F908F90DA
:102DE0000895EF92FF920F931F93CF93DF93EC011F
:102DF000162F0AE08881882309F457C0813009F032
:102E00004FC08981813041F47E0182E0E80EF11CDF
:102E10008A810E942D0609C0823049F47E01E2E0D9
:102E2000EE0EF11C8A810E943F05E7012DC0833020
:102E300041F47E01F2E0EF0EF11C8A810E94C4058C
:102E4000F4CF843011F021961FC02A81229680E0B1
:102E500090E030E0205331092A30310558F4089FC2
:102E6000A001099F500D1124C901840F951F2196BF
:102E70002881EFCF009741F0EFE9FFE03197F1F7BC
:102E800000C000000197F6CF812F90E0009759F025
:102E9000EFE9FFE03197F1F700C000000197F6CFAE
:102EA000612F0E943F162196A5CFCDB7DEB7E6E091
:102EB0000C94DF230F931F93CF93DF93C42FD22F54
:102EC000FC0185818823B1F040939F020E94131C6E
:102ED00090939E0280939D0280E28C0F883008F0D0
:102EE0004DC0C77081E001C0880FCA95EAF70E9403
:102EF000370644C080919F02481330C080919D02E4
:102F000090919E020E942B1C883C910538F510E29E
:102F10001D0FCD17B9F080E28C0F883040F4C770D8
:102F200081E001C0880FCA95EAF70E943E0618307A
:102F300010F581E09D2F977001C0880F9A95EAF7F0
:102F40000E943706802F0E942D061830B8F4D770E3
:102F500081E001C0880FDA95EAF70AC080E28C0FA1
:102F6000883060F4C77081E001C0880FCA95EAF725
:102F70000E943E0603C0802F0E942D06DF91CF9154
:102F80001F910F9108950F93FC01E851FC47E73022
:102F9000F10590F5CB01EC57FF4F0C94AA2306E204
:102FA00021EE41EE6AE17CE723C007E225EE45EE23
:102FB0006BE17CE71DC006E221EE40EE68E17CE7B4
:102FC00017C007E225EE44EE69E17CE711C006E296
:102FD00021EE42EE6CE17CE70BC007E225EE46EE07
:102FE0006DE17CE705C008E221E045EE6EE17CE79B
:102FF0000E945A1780E008C0FB018581882319F0E0
:1030000010929F0201C081E00F9108951F93CF930A
:10301000DF9387372CE7920721F088379C4759F0D8
:1030200031C0FB01C581CC2319F00E94481809C0AA
:103030000E94481818C0FB01C581CC2391F00E9462
:103040004B180E94EF080E944E18D82F0E944B1870
:10305000C82F0E9448184D2F6C2F0E94190AC0E0FB
:1030600012C00E944B180E94FB080E944E18182F95
:103070000E944B18D82F0E944818412F6D2F0E9494
:10308000190A01C0C1E08C2FDF91CF911F910895E3
:1030900080910601089580910501089580910401B1
:1030A000089584E290E00E940424853281F485E250
:1030B00090E00E940424813051F486E290E00E9466
:1030C000042491E0843109F090E0892F01C080E070
:1030D00081700895CF93C82F811102C06FEF01C096
:1030E00065E284E290E00E942224C11102C06FEFE9
:1030F00001C061E085E290E00E942224C11102C07B
:103100006FEF01C064E186E290E00E942224CF913B
:103110000895089587E290E00E940424682F70E0EB
:1031200080E090E008950895CF93C62F0E949318F1
:103130006C2F87E290E00E942224CF91089580E0D6
:103140000E946A1860E070E0CB010E9494180E940F
:10315000E5130E94981481E00E946A1808950E9465
:1031600089180E948A180E9493180E945118811190
:1031700002C00E949F18089508959C01FB0185815B
:10318000882351F0A90157574038510530F4C9013F
:103190000E94A81480E0089581E008952FEFFC01BB
:1031A000208308950E94CE18089580E00895A0E03D
:1031B000B0E0EDEDF8E10C94BF23EC01D62E0E94B7
:1031C000D5188111BEC0E8818E2F90E0FC013197A7
:1031D000E331F10508F0AFC0E557FF4F0C94AA2387
:1031E00019828CE06BC08981823089F030F48130A3
:1031F00009F0A1C00E941F1C0CC0833079F08430FC
:1032000009F099C01A821B821C821D8296C00E94FE
:103210008A189A838B837C836D838FC0CA807E01DA
:1032200000E010E0AC2CB12CC501800F911F0C9771
:1032300008F083C08C2D800F0E940A12F70193833F
:1032400084830F5F1F4FF2E0EF0EF11C0E3011056B
:1032500059F773C08981823039F0853009F06BC02D
:103260008A810E94BC1869C06A817B818C819D81A2
:103270000E94B0230E94941860C04B816A818981AA
:103280000E94A9139C838D8358C02C813D813227D5
:10329000232732274B816A8189810E94CA134DC03E
:1032A0000E94E5134AC06D2DCE010E94D21845C080
:1032B0000E94511424C00E94531499838A833DC0F4
:1032C0006B8170E089819A81AE014C5F5F4F9827D6
:1032D000892798270E94561430C06B8170E089813D
:1032E0009A81AE014C5F5F4F9827892798270E94EB
:1032F000781423C00E94981420C00E9496138983DA
:103300001CC06B8170E089819A81AE014C5F5F4F78
:103310009827892798270E9403140FC06B8170E0BB
:1033200089819A81AE014C5F5F4F98278927982742
:103330000E94251402C08FEF88836D2DCE010E945C
:10334000D81CCDB7DEB7EAE00C94DB239093A5023E
:103350008093A4020895E091A402F091A502309711
:1033600029F00190F081E02D0995089580E00895FD
:103370000E94AB190895E091A402F091A502309744
:1033800021F00280F381E02D09950895E091A402D7
:10339000F091A502309739F026E0DC012C930480EF
:1033A000F581E02D09950895A3E0B0E0EAEDF9E19B
:1033B0000C94C7232091A2023091A3022817390749
:1033C000A1F09093A3028093A202E091A402F09155
:1033D000A502309751F023E029839B838A830084E0
:1033E000F185E02DCE01019609952396E2E00C943B
:1033F000E323A3E0B0E0EFEFF9E10C94C7232091C1
:10340000A0023091A10228173907A1F09093A102E0
:103410008093A002E091A402F091A502309751F0B0
:1034200024E029839B838A830084F185E02DCE01EB
:10343000019609952396E2E00C94E323CF93DF9362
:10344000C0910201D091030122960E94621B81303B
:1034500059F48091AF0287FF07C0C0910001D0915D
:10346000010122969EE101C096E080E0915028F093
:1034700029912223D9F38F5FF9CFDF91CF9108955E
:10348000CF93882329F1C82F0E94621B813011F548
:103490008091AF0287FF1EC08C2F869586958695FA
:1034A0008E31B0F4E0910001F0910101E80FF11DBF
:1034B0002281822F90E0C77021E030E002C0220F0D
:1034C000331FCA95E2F72823392381E0232B89F49F
:1034D00080E00FC08091020190910301FC013296BF
:1034E00008962191C21721F0E817F907D1F7F0CF1C
:1034F00081E0CF9108959C01FC0132969FEF80E01E
:103500004191461789F09F3F19F4411101C0982F4E
:103510008F5F8630A9F79F3F39F0F901E90FF11D60
:1035200097FDFA956283089508959C012A5F3F4FA5
:10353000FC014281461301C0128201968217930753
:10354000B9F70895262F2695269526952E3168F4ED
:10355000FC01E20FF11D677021E030E001C0220F95
:103560006A95EAF78281282B22830895262F2695D3
:10357000269526952E3170F4FC01E20FF11D67703F
:1035800021E030E001C0220F6A95EAF720958281A0
:10359000282322830895CF93C82F0E94621B6C2F8B
:1035A000813059F48091AF0287FF07C080910001FC
:1035B000909101010E94A21A06C08091020190918F
:1035C00003010E947B1ACF910895CF93C82F0E94C8
:1035D000621B6C2F813059F48091AF0287FF07C0C6
:1035E00080910001909101010E94B61A06C080915D
:1035F0000201909103010E94951ACF9108950E94B3
:10360000621B813059F48091AF0287FF07C0E091BF
:103610000001F091010132968EE106C0E0910201B5
:10362000F0910301329686E0DF011D928A95E9F759
:10363000089508950E94191B089583E080930A015C
:1036400060910701709108018091090190910A0130
:103650000E941A1B0895811102C081E001C082E01E
:1036600080930A016091070170910801809109011E
:1036700090910A010E941A1B08950E942B1B089525
:1036800081E080930A0160910701709108018091A7
:10369000090190910A010E941A1B08950E94401B83
:1036A000089591E0811101C090E09093090160912B
:1036B0000701709108018091090190910A010E940F
:1036C0001A1B089580910901089580930801609163
:1036D0000701709108018091090190910A010E94EF
:1036E0001A1B089580910801089580930701609145
:1036F0000701709108018091090190910A010E94CF
:103700001A1B089580910701089508950E94851B52
:1037100008950E94861B08950E94851B08950E94AB
:10372000851B08950E94851B0895CF930E948F1BCF
:103730000E94DE120E948C1BC0E08C2F0E940A1295
:10374000892B29F4CF5FCC30C1F780E001C081E044
:10375000CF91089585B7806885BF85B7806885BF9C
:1037600008951F920F920FB60F9211248F939F937B
:10377000AF93BF938091A602811113C08091E102A3
:103780009091E202A091E302B091E4024196A11D62
:10379000B11D8093E1029093E202A093E302B09303
:1037A000E402BF91AF919F918F910F900FBE0F9048
:1037B0001F9018958091E902843031F10E94C10474
:1037C0001092A60220E488E190E00FB6F894A89544
:1037D000809360000FBE2093600083B7817F846078
:1037E00083BF83B7816083BF7894889583B78E7FCA
:1037F00083BF0FB6F894A89580916000886180938C
:103800006000109260000FBE08950E9477080E9429
:10381000C604089582E084BD93E095BD9AEF97BDFC
:1038200080936E0008952FB7F8948091E1029091F3
:10383000E202A091E302B091E4022FBF08952FB7F6
:10384000F8946091E1027091E2028091E30290911C
:10385000E4022FBF08959C014FB7F8948091E102D4
:103860009091E202A091E302B091E4024FBF821B6B
:10387000930B089578941F920F920FB60F92112414
:103880008F939F93AF93BF938091E1029091E20257
:10389000A091E302B091E4020196A11DB11D8093B5
:1038A000E1029093E202A093E302B093E402BF919D
:1038B000AF919F918F910F900FBE0F901F90189511
:1038C00081E08093E00080E28093D8001092C900EC
:1038D0008FE19EE40197F1F700C0000087E090EBD4
:1038E000DC018093F2029093F302A093F402B09370
:1038F000F5029CE088E10FB6F894A89580936000EB
:103900000FBE90936000FFCF9CE088E10FB6F89463
:10391000A895809360000FBE90936000FFCF08953C
:103920009B019091E9029430F1F48F708093E9004B
:103930008FEF9091E800815095FD06C095ED9A9526
:10394000F1F700008111F5CF8091E80085FF0BC0F1
:10395000BA01C90140E050E00E94D71E8091E80002
:103960008E778093E800089543E050E0BC0184E046
:103970000E94901C089540E250E0BC0184E00E9447
:10398000901C0895CF93DF93EC010E94621B48E0E6
:1039900050E0BE0181E00E94901C88E0FE01A7EA91
:1039A000B2E001900D928A95E1F7DF91CF910895F1
:1039B000603231F4BC0140E250E082E00E94901C91
:1039C0000895A0E2B0E0E7EEFCE10C94C7238091FB
:1039D000E902843011F583E08093E9008091E800EA
:1039E00082FF1BC08091E80085FF0AC040E050E0E4
:1039F00060E270E0CE0101960E941C1F91E001C0C0
:103A000090E08091E8008B778093E800992329F07B
:103A100060E2CE0101960E94D718A096E2E00C94D5
:103A2000E3238091E802811109C00E94A7200E942F
:103A300004218091E20084608093E2000895109256
:103A4000E80208950E944E1B81E00E94511B0895D8
:103A50006091E50281E0611101C080E00E941D1BC0
:103A600008959091E90281E0943009F080E060913E
:103A7000E5020E942B1B089542E061EC81E00E9468
:103A8000202042E261EC84E00E94202042E261ECCE
:103A900082E00E94202042E260EC83E00E9420202D
:103AA0009091E90281E0943009F080E06091E502B4
:103AB0000E943D1B08958091EB02833009F463C09E
:103AC00030F4813071F0823009F49DC008958A305D
:103AD00009F489C08B3009F46EC0893009F0ABC09D
:103AE00020C08091EA02813A09F0A5C08091E800E7
:103AF000877F8093E8008091EE029091EF02892BFE
:103B000021F468E087EA92E003C060E080E090E0A2
:103B100070E00E94611F8091E8008B778093E8003D
:103B200008958091EA02813209F085C08091EE0209
:103B30009091EF02009719F0029709F07CC08091F4
:103B4000E800877F8093E8008091E80082FD05C04F
:103B50008091E9028111F8CF6EC02091F30080912D
:103B6000F20090E0922B029731F48091F1008130C5
:103B700011F0863021F48091F1000E94651B809144
:103B8000E8008B7754C08091EA02813A09F053C073
:103B90008091EE029091EF02892B09F04CC0809148
:103BA000E800877F8093E8008091E80080FFFCCFE9
:103BB0000E94621B37C08091EA028132E1F5809158
:103BC000EE029091EF02892BB1F58091E800877F9A
:103BD0008093E8000E9455208091EC020E94511BC6
:103BE0000E94770808958091EA02813221F5809140
:103BF000E800877F8093E8000E9455208091ED02C5
:103C00000E94751B08958091EA02813AA1F4809187
:103C1000E800877F8093E8008091E80080FFFCCF78
:103C20000E94821B8093F1008091E8008E77809340
:103C3000E8000E945520089584B7877F84BF0FB69F
:103C4000F894A8958091600088618093600010923C
:103C500060000FBE90E080E80FB6F894809361009A
:103C6000909361000FBE0E94401B08950E94A72000
:103C70000E940421E2EEF0E08081846080837894E9
:103C80000E948F2308958BE091E00E94A619089569
:103C90008091E9028530A9F48091E902853079F4B8
:103CA0000E94DA1B0E94951B8823B1F38091E702E2
:103CB000882391F30E94C11E0E947708EDCF0E94D5
:103CC000051C089508959A014091F0025091F10267
:103CD0000E946B1E0895492F552743305105C9F0A6
:103CE00060F44130510581F04230510509F041C086
:103CF0008BE590E046E855E040C041325105E1F0E7
:103D00004232510531F135C082E190E041EE55E09B
:103D100034C099278130910549F028F0029749F580
:103D2000E0E6F5E005C0E2E8F5E002C0EEE6F5E029
:103D3000849190E0AF0121C063307105D0F4660F2B
:103D4000771FFB01EB55FE4F4081518189E090E0E8
:103D500014C06330710568F4FB01EE0FFF1FE156DC
:103D6000FE4F40815181FB01E456FE4F808190E07F
:103D700004C080E090E040E050E0F90151834083CE
:103D8000089580E189BD82E189BD09B400FEFDCFBF
:103D90008091D8008F7D8093D8008091E000826070
:103DA0008093E0008091E00081FDFCCF0895A0E0C9
:103DB000B0E0EDEDFEE10C94C123EC018B017A0142
:103DC0000E947420811133C0E114F10439F0F7012D
:103DD00080819181081B190BC80FD91FC12CD12CD0
:103DE0000115110519F18091E80085FD16C080913B
:103DF000E8008E778093E800E114F10449F0F701C0
:103E000080819181C80ED91ED182C08285E00FC009
:103E10000E947420882321F30AC089918093F100C5
:103E200001501109FFEFCF1ADF0ADACF80E0CDB7DA
:103E3000DEB7E8E00C94DD23A0E0B0E0E2E2FFE1D1
:103E40000C94C123EC018B017A010E947420811132
:103E500033C0E114F10439F0F70180819181081B2E
:103E6000190BC80FD91FC12CD12C0115110519F13F
:103E70008091E80085FD16C08091E8008B778093E3
